:10044F00E4750F80750E25F50DF50C7510407511BF
:10045F0030751210FF7E247DF4FC1201DFE4FD7F66
:04046F00010204DDA5
:100473007D087F0512052F7D01E4FF12042AE4FDA8
:0A0483007F011204B97F0102050F8A
:1003960012044F120473D2AF12053E3000FDC200A4
:1003A60012048DEEFF1205463002FDC20212048DC4
:1003B6001205463002FDC202E4F513F514C3E51436
:1003C6009490E513940150D0E4F515F5160516E55D
:1003D6001670020515B4F4F5E515B401F00514E53B
:0703E6001470DA051380D644
:06052200C100C102C1018D
:0300030002054CA7
:01054C00327C
:03000B0002054D9E
:01054D00327B
:0300130002054E95
:01054E00327A
:03001B0002054F8C
:01054F003279
:0300230002033E97
:10033E00C0E0C0F0C083C082C0D075D000C000C085
:10034E0001C002C003C004C005C006C0077F021270
:10035E000534EF60097F02120539D202800F7F014A
:10036E00120534EF60077F01120539D201D007D094
:10037E0006D005D004D003D002D001D000D0D0D00A
:08038E0082D083D0F0D0E032F0
:03002B000205507B
:010550003278
:030033000203EDD8
:1003ED00C0E0C0F0C083C082C0D075D000C000C0D6
:1003FD0001C002C003C004C005C006C007120542FB
:10040D00D200D007D006D005D004D003D002D00141
:0D041D00D000D0D0D082D083D0F0D0E0321B
:03003B000205516A
:010551003277
:0300430002055261
:010552003276
:03004B0002055358
:010553003275
:030053000205544F
:010554003274
:1004EF00E4F5ADF5ABF5AAF5AEF5AFC2AEC2BE22DF
:05052F00EF4DF5AA22CA
:10042A00E5AD54E04FF5ADA8077401088002C33367
:10043A00D8FCFEEFC3941F500BED7005EEF452ABDF
:04044A0022EE42ABB1
:01044E00228B
:0B050F00EF700453AD7F2243AD80224B
:04053E0043AD402267
:10048D00AFAFEF75F010A4FFE5AEC4540F7C002F95
:05049D00FFEC35F0FE4C
:0104A2002237
:1004B900EF7004C2AE8002D2AEED7003C2BE22D28A
:0204C900BE2251
:06052900E5AD5420FF22A5
:0405420053ADDF22B4
:1004FF00538FEFE4F59853877F53A8EF53B8EF224C
:08051A00E58F54DF4FF58F223D
:1001DF008F0B8E0A8D098C08E598542F4510451208
:1001EF00F598E5107031FFFEFDFCAB0FAA0EA90DBF
:1001FF00A80CC31201CE700453877F22E47F01FE47
:10020F00FDFCAB0FAA0EA90DA80CC31201CE600303
:10021F000202A343878022E5C854CF4511F5C8E5F4
:10022F00117036AB0FAA0EA90DA80CAF0BAE0AAD0D
:10023F0009AC0812013CE4FB7A01F9F812013C8F7A
:10024F008DAB0FAA0EA90DA80CAF0BAE0AAD09AC62
:10025F000812013C8F8BC28E22E51164307035ABD2
:10026F000FAA0EA90DA80CAF0BAE0AAD09AC081260
:10027F00013CE4FB7A01F9F812013C8FCBAB0FAADA
:10028F000EA90DA80CAF0BAE0AAD09AC0812013CBC
:05029F008FCAD2CA2243
:030546008F992268
:03054900AF992245
:0404CB00AD07AC06C7
:0D04CF00EC600543980880035398F78D9961
:0104DC0022FD
:1004A300E598540475F040A4AD997C002DFFEC351C
:0504B300F0FE5398FB70
:0104B8002221
:1004DD00EF7004C2AC8002D2ACED7003C2BC22D26C
:0204ED00BC222F
:05053400E5985FFF22C5
:05053900EFF4529822CE
:030000000202A455
:1002A40078FFE4F6D8FD9000007F007E01E4F0A31F
:0A02B400DFFCDEFA7581200202F97A
:1002BE00020396E493A3F8E493A34003F68001F2BD
:1002CE0008DFF48029E493A3F85407240CC8C33341
:1002DE00C4540F4420C8834004F456800146F6DF10
:1002EE00E4800B0102040810204080900522E47E79
:1002FE00019360BCA3FF543F30E509541FFEE49305
:10030E00A360010ECF54C025E060A840B8E493A3CB
:10031E00FAE493A3F8E493A3C8C582C8CAC583CAF6
:10032E00F0A3C8C582C8CAC583CADFE9DEE780BEAE
:0105280000D2
:1001000075F008758200EF2FFFEE33FECD33CDCCB6
:1001100033CCC58233C5829BED9AEC99E582984039
:100120000CF582EE9BFEED9AFDEC99FC0FD5F0D616
:10013000E4CEFBE4CDFAE4CCF9A88222B800C1B940
:100140000059BA002DEC8BF084CFCECDFCE5F0CB7E
:10015000F97818EF2FFFEE33FEED33FDEC33FCEBB7
:1001600033FB10D703994004EB99FB0FD8E5E4F972
:10017000FA227818EF2FFFEE33FEED33FDEC33FC5F
:10018000C933C910D7059BE99A4007EC9BFCE99A53
:10019000F90FD8E0E4C9FAE4CCFB2275F010EF2F98
:1001A000FFEE33FEED33FDCC33CCC833C810D70798
:1001B0009BEC9AE899400AED9BFDEC9AFCE899F8D3
:0E01C0000FD5F0DAE4CDFBE4CCFAE4C8F92266
:1001CE00EB9FF5F0EA9E42F0E99D42F0E89C45F087
:0101DE0022FE
:00000001FF
